:100000009AC00000B3C00000B1C00000AFC0000043
:10001000ADC00000ABC00000A9C00000A7C0000038
:10002000A5C00000A3C00000A1C00000DCC3000008
:100030009DC000009BC0000099C0000097C0000058
:1000400095C0000093C0000091C000008FC0000068
:100050008DC000008BC0000089C00000E7C0000018
:1000600085C0000083C0000081C000007FC0000088
:100070007DC000007BC0000079C0000077C0000098
:1000800075C0000073C0000071C000006FC00000A8
:100090006DC000006BC0000005010906A1017501DB
:1000A0009508050719E029E715002501810295014A
:1000B0007508810395057501050819012905910247
:1000C00095017503910395067508150026E700054F
:1000D00007190029E78100C0120110010000000883
:1000E000EB0342200000010200010902220001018D
:1000F00000C03209040000010301010009211101BF
:1001000000012240000705810308000A04030904D6
:100110001003410072006400750069006E006F00FA
:10012000000012034B006500790062006F0061005F
:1001300072006400000011241FBECFEFD2E0DEBFCA
:10014000CDBF11E0A0E0B1E0EEEAFFE002C0059013
:100150000D92AE30B107D9F711E0AEE0B1E001C0C9
:100160001D92AE3AB107E1F7F4D01FC749CF089509
:10017000089580910B0190910C01009729F001974F
:1001800090930C0180930B0108950F931F93CF93CD
:10019000DF93E8018FB7F8949091A3018FBF983057
:1001A00048F1AEE0B1E06FE171E0E091A101F091C2
:1001B000A2014191F093A201E093A101EF59F14016
:1001C00021F47093A2016093A1019FB7F8948091EC
:1001D000A30181508093A3019FBF4D9381E0A6317D
:1001E000B80719F7909116018091C80085FFFCCFE0
:1001F0009093CE0040E050E0F901E40FF51FDA01E2
:10020000A25FBE4F8C9180834F5F5F4F4830510596
:1002100099F75983488380E0DF91CF911F910F9127
:100220000895F90180818093160108951F920F921D
:100230000FB60F9211242F938F939F93EF93FF93F9
:100240009091CE008EB38430F1F4E0919F01F09153
:10025000A0019083E0919F01F091A001CF01019650
:100260009093A00180939F018F59914021F48FE1D9
:1002700091E0928381839FB7F8948091A3018F5F6F
:100280008093A3019FBFFF91EF919F918F912F9139
:100290000F900FBE0F901F90189580E091E042C51F
:1002A00080E091E00ED5E2EEF0E080818460808312
:1002B00008959F92AF92BF92CF92DF92EF92FF92FA
:1002C0000F931F9384B7877F84BF28E10FB6F894FC
:1002D00020936000109260000FBE4CECA42EB12C55
:1002E00087E690E0F501918380833AECC32ED12C10
:1002F00096E0992EF601908208EC10E0F801108249
:1003000089ECE82EF12CF7012083539A5A9A60D297
:1003100084E085BD5F9A579AF7011082F801108238
:10032000F60110828FEC90E0F50191838083F60155
:10033000908282E0F801808388E9F70180831F9131
:100340000F91FF90EF90DF90CF90BF90AF909F9074
:100350000895AFDF2FB7F8948FE191E09093A0015B
:1003600080939F019093A2018093A1012FBF789465
:1003700080E091E0EDD3DAD3FBCFDA019330B1F036
:10038000943028F4913041F0923079F50AC09132DE
:1003900011F1923251F524C0E8EDF0E022E130E0B5
:1003A00028C0EAEEF0E022E230E023C0813049F0DC
:1003B000813018F08230C9F40AC0ECE0F1E0849199
:1003C00003C0E0E1F1E08491282F30E012C0E2E2C6
:1003D000F1E08491F9CFECEFF0E029E030E009C0E2
:1003E000E8E9F0E020E430E004C0E0E0F0E020E004
:1003F00030E0ED93FC93C901089528E030E040E03F
:1004000003C04F5F220F331F28173907D0F3842F03
:100410008295807F08958093E9008091EB00816050
:100420008093EB001092ED006093EC004093ED00A0
:100430008091EE00881F8827881F08951092F4008D
:1004400090E09093E9001092F0001092E800109272
:10045000ED008091EB008E7F8093EB009F5F9530E5
:1004600081F708958091A60188238CF403C08EB390
:100470008823B1F08091E80082FFF9CF8091E800F5
:100480008B778093E80008958EB3882349F080919C
:10049000E80080FFF9CF8091E8008E778093E80034
:1004A000089594E68091EC0080FF05C08091E800FB
:1004B00080FF05C023C08091E80082FD1FC08EB37D
:1004C000882311F482E008958EB3853011F483E01F
:1004D00008958091EB0085FF02C081E0089580912E
:1004E000E10082FFDFCF8091E1008B7F8093E1000C
:1004F000992311F484E008959150D4CF80E00895B9
:10050000DF92EF92FF920F931F93CF93DF93182FF9
:10051000092FEB017A01C5DFD82E882319F5812F29
:10052000902F9C0189011CC08091E80085FD12C0BC
:100530008091E8008E778093E800E114F10431F0B7
:10054000F7010995813011F485E00DC0AADF8823F9
:1005500039F009C0F80181918F018093F100219752
:10056000209711F78D2DDF91CF911F910F91FF9063
:10057000EF90DF9008959C014091AC015091AD0146
:100580004617570718F4F90120E038C061157105C6
:1005900011F0AB01F8CF8091E8008E778093E800EE
:1005A00040E050E0F0CF8091E80083FF02C081E09E
:1005B00008958091E80082FD2DC08EB3882381F1DB
:1005C0008EB3853079F18091E80080FF17C090915B
:1005D000F20006C081918093F100415050409F5F2E
:1005E0004115510511F09830A8F320E0983009F436
:1005F00021E08091E8008E778093E8004115510555
:1006000091F6222381F606C08EB3882349F08EB37B
:10061000853041F08091E80082FFF6CF80E00895B8
:1006200082E0089583E008959C014091AC015091CF
:10063000AD014617570710F490E03BC061157105F6
:1006400011F0AB01F9CF8091E8008E778093E8003C
:1006500040E050E0F1CF8091E80083FF02C081E0EC
:1006600008958091E80082FD30C08EB3882399F10F
:100670008EB3853091F18091E80080FF1AC080919F
:10068000F20009C0F9012F5F3F4FE491E093F100C0
:10069000415050408F5F4115510511F0883090F363
:1006A00090E0883009F491E08091E8008E778093A3
:1006B000E8004115510579F6992369F606C08EB315
:1006C000882349F08EB3853041F08091E80082FFA5
:1006D000F6CF80E0089582E0089583E008959C01BC
:1006E0006115710529F48091E8008B778093E8000B
:1006F000F90120C08091E80083FF02C081E00895E5
:100700008EB3882339F18EB3853031F18091E800C2
:1007100082FFF0CF06C08091F1008193615070405C
:1007200021F08091F2008823B1F78091E8008B7767
:100730008093E80061157105E9F606C08EB3882341
:1007400049F08EB3853041F08091E80080FFF6CF0C
:1007500080E0089582E0089583E008953ED040D07F
:100760001EBA1092A40184E089BD89B5826089BD5A
:1007700009B400FEFDCF8091D800982F9F77909309
:10078000D80080688093D800809163008E7F80932A
:1007900063008091D8008F7D8093D8008091E00025
:1007A0008E7F8093E0008091E1008E7F8093E10056
:1007B0008091E20081608093E2008091E100877F78
:1007C0008093E1008091E20088608093E2000895C8
:1007D000C5DF81E08093A50108951092E20008959D
:1007E0001092E10008951F920F920FB60F921124FC
:1007F0002F933F934F935F936F937F938F939F9329
:10080000AF93BF93EF93FF938091E10080FF1BC0F4
:100810008091E20080FF17C08091E1008E7F80937D
:10082000E1008091E2008E7F8093E2008091E200FF
:1008300080618093E2008091D80080628093D8002C
:1008400019BC1EBA95DC8091E10084FF29C080911B
:10085000E20084FF25C084E089BD89B5826089BD3E
:1008600009B400FEFDCF8091D8008F7D8093D80021
:100870008091E1008F7E8093E1008091E2008F7E85
:100880008093E2008091E20081608093E200809199
:10089000A401882311F481E001C084E08EBB67DCF1
:1008A0008091E10083FF22C08091E20083FF1EC09F
:1008B0008091E100877F8093E10082E08EBB1092FF
:1008C000A4018091E1008E7F8093E1008091E2009D
:1008D0008E7F8093E2008091E20080618093E2004D
:1008E000ADDD80E060E042E096DD1FD18091E10067
:1008F00082FF0AC08091E20082FF06C08091E10081
:100900008B7F8093E10035DCFF91EF91BF91AF9138
:100910009F918F917F916F915F914F913F912F9117
:100920000F900FBE0F901F9018951F93DF93CF93DA
:1009300000D0CDB7DEB7E6EAF1E08091F100819317
:1009400081E0EE3AF807C9F78091A6019091A701DE
:10095000953009F46DC0963040F4913081F19130BA
:1009600070F0933009F0CCC02AC0983009F49EC0D2
:10097000993009F4ADC0963009F0C2C078C0803813
:1009800009F4BFC0823809F0BBC08091AA0187700A
:100990008093E9008091EB001092E9002091E8003B
:1009A000277F2093E80090E025E0969587952A958B
:1009B000E1F781708093F1001092F10082C08823EA
:1009C00019F0823009F09CC08F71823009F099C013
:1009D0008091A801882331F52091AA01277009F49C
:1009E00090C02093E9008091EB0080FF8AC0933093
:1009F00021F48091EB00806213C08091EB00806154
:100A00008093EB0081E090E002C0880F991F2A9547
:100A1000E2F78093EA001092EA008091EB00886090
:100A20008093EB001092E9008091E800877F4CC032
:100A3000882309F065C01091A8018091E800877FA4
:100A40008093E8000FDD04C08EB3882309F459C0F9
:100A50008091E80080FFF8CF812F8F7711F492E02A
:100A600001C093E09EBB80688093E3004AC0805839
:100A7000823008F045C08091A8019091A901609151
:100A8000AA01AE014F5F5F4F78DCBC010097C9F14E
:100A90008091E800877F8093E80089819A81C4DD96
:100AA0008091E8008B778093E8002BC0803841F577
:100AB0008091E800877F8093E8008091A401809373
:100AC000F1008091E8008E778093E800CBDC19C0BC
:100AD0008823B1F49091A801923098F48091E800B5
:100AE000877F8093E8009093A401BCDC8091A401EF
:100AF000882311F483E001C084E08EBBD1DB01C008
:100B0000CCDB8091E80083FF0AC08091EB0080621B
:100B10008093EB008091E800877F8093E8000F903E
:100B20000F90CF91DF911F91089508951F938EB379
:100B3000882361F01091E9001092E9008091E800AB
:100B400083FF01C0F2DE17701093E9001F91089532
:100B50004F925F926F927F928F929F92AF92BF92CD
:100B6000CF92DF92EF92FF920F931F93DF93CF9379
:100B700000D00F92CDB7DEB77C016DB67EB68EB3D6
:100B8000843009F085C0F70181818093E90080916C
:100B9000E80085FF7DC05DB64EB647818DB79EB734
:100BA000841B91090FB6F8949EBF0FBE8DBF0DB781
:100BB0001EB70F5F1F4F19821B821A82C02E912E03
:100BC000C80160E070E050E0E9D1C701BE016F5F8D
:100BD0007F4F40E098018E010E5F1F4FD6DA882EBE
:100BE000F70181859285892B19F4AA24BB240BC0B7
:100BF00020E0F70183859485892B09F021E081E0CD
:100C00002827A22EBB24F7010581168101151105A5
:100C100011F4DD2412C04A815B818C2D992DB8011D
:100C2000A7D1DD24009711F0DD24D394F70147818B
:100C3000C8016C2D792D50E0A8D18A819B81892B28
:100C4000F9F0882021F4DD2011F4AB28C9F0F70178
:100C5000818592859487838781818093E90089814A
:100C6000882311F08093F1006A817B818C2D992D6E
:100C700040E050E045DC8091E8008E778093E8000A
:100C8000852D942D9C010FB6F8943EBF0FBE2DBF4D
:100C90000FB6F8947EBE0FBE6DBE0F900F900F90F2
:100CA000CF91DF911F910F91FF90EF90DF90CF9048
:100CB000BF90AF909F908F907F906F905F904F907C
:100CC00008950F931F93CF93DF93DC010896FC01E7
:100CD00085E0EF0119928A95E9F781E018968C93E7
:100CE000189784EF91E01A969C938E931997129619
:100CF0002D913C91139711960C91119714968C910C
:100D0000882311F410E001C014E0C90176DB182B30
:100D10001260802F61EC412F7EDBDF91CF911F911C
:100D20000F9108956F927F928F929F92AF92BF9290
:100D3000CF92DF92EF92FF920F931F93DF93CF93A7
:100D400000D00F92CDB7DEB74C016DB67EB6809164
:100D5000E80083FFF6C0F401808190E02091AA01B1
:100D60003091AB012817390709F0EBC08091A7013A
:100D7000833009F498C0843030F4813071F08230CF
:100D800009F0DFC0C6C08A3009F4ACC08B3009F46A
:100D900097C0893009F0D5C04FC08091A601813A33
:100DA00009F0CFC0ADB6FEB68091E800877F809392
:100DB000E8001B821A828091A8011091A901898301
:100DC000F40147818DB79EB7841B91090FB6F89443
:100DD0009EBF0FBE8DBFCDB6DEB60894C11CD11C20
:100DE000EC2CBD2CC60160E070E050E0D7D0115073
:100DF000C401BE016F5F7F4F412F96018E010E5FD0
:100E00001F4FC3D9F401258136812115310529F001
:100E10004781C901B60150E0B8D01092E9006A815B
:100E20007B818E2D9B2DA7DB8091E8008B778093B3
:100E3000E8002A2D3F2D31C08091A601813209F0B2
:100E400080C0AEB68091E800877F8093E800009173
:100E5000AC011091AD01C090A801D090A9018DB74F
:100E60009EB7801B910B0FB6F8949EBF0FBE8DBF2F
:100E7000EDB6FEB60894E11CF11CC701B8012FDCE9
:100E8000DA94C4016C2D4D2D9701CBD98091E800E7
:100E90008E778093E800262D3A2D0FB6F8943EBF4A
:100EA0000FBE2DBF4EC08091A601813A09F049C006
:100EB0008091E800877F8093E800F401808539C045
:100EC0008091A601813209F03CC08091E800877FC3
:100ED0008093E80090E08091A801811191E0F401F5
:100EE00090872EC08091A601813259F58091E8004B
:100EF000877F8093E8008091A8019091A90180707C
:100F000036E0969587953A95E1F7F40192878187C7
:100F100017C08091A601813AA1F48091E800877FF3
:100F20008093E800F4018185928596958795969542
:100F300087958093F1008091E8008E778093E80098
:100F400091DA0FB6F8947EBE0FBE6DBE0F900F9073
:100F50000F90CF91DF911F910F91FF90EF90DF9055
:100F6000CF90BF90AF909F908F907F906F9008959B
:100F7000FB01DC0104C08D910190801921F44150E6
:100F80005040C8F7881B990B0895FB01DC0102C093
:100F900001900D9241505040D8F70895DC0101C0F6
:0E0FA0006D9341505040E0F70895F894FFCF54
:0E0FAE0000010800001701080000000000000C
:00000001FF
